:020000040000FA
:040800004DEF0BF0BD
:1008100003B276EF05F0F2B494EF05F09EB09CEFD2
:1008200005F09EB2A4EF05F0F2A81AEF04F0F2B2C0
:1008300025EF04F0F2A620EF04F0F2B022EF04F06E
:10084000FCEF0AF0F296F290FF00CD90F2929EA09B
:100850002FEF04F00101533F2FEF04F0542BAEC1F2
:10086000B2F1AFC1B3F1B0C1B4F1B1C1B5F1AAC138
:10087000AEF1ABC1AFF1ACC1B0F1ADC1B1F1A6C148
:10088000AAF1A7C1ABF1A8C1ACF1A9C1ADF1A2C158
:10089000A6F1A3C1A7F1A4C1A8F1A5C1A9F19EC168
:1008A000A2F19FC1A3F1A0C1A4F1A1C1A5F19AC178
:1008B0009EF19BC19FF19CC1A0F19DC1A1F196C188
:1008C0009AF197C19BF198C19CF199C19DF1CECF4E
:1008D00096F1CFCF97F153C198F154C199F1CF6AF6
:1008E000CE6A0101536B546B9E90CD800FBC0F8E6E
:1008F0000FBA7EEF04F00F8AFCEF0AF00F8C0FBEE8
:10090000BAEF04F096C19AF197C19BF198C19CF19E
:1009100099C19DF19AC19EF19BC19FF19CC1A0F12B
:100920009DC1A1F19EC1A2F19FC1A3F1A0C1A4F1FB
:10093000A1C1A5F1A2C1A6F1A3C1A7F1A4C1A8F1CB
:10094000A5C1A9F1A6C1AAF1A7C1ABF1A8C1ACF19B
:10095000A9C1ADF1AAC1AEF1ABC1AFF1ACC1B0F16B
:10096000ADC1B1F1AEC1B2F1AFC1B3F1B0C1B4F13B
:10097000B1C1B5F101015E6B5F6B606B616B96514C
:100980005E2797515F2398516023995161239A51B3
:100990005E279B515F239C5160239D5161239E5193
:1009A0005E279F515F23A0516023A1516123A25173
:1009B0005E27A3515F23A4516023A5516123A65153
:1009C0005E27A7515F23A8516023A9516123AA5133
:1009D0005E27AB515F23AC516023AD516123AE5113
:1009E0005E27AF515F23B0516023B1516123B251F3
:1009F0005E27B3515F23B4516023B5516123D89072
:100A00000101613360335F335E33D890010161339C
:100A100060335F335E33D8900101613360335F33FD
:100A20005E3300C10CF101C10DF102C10EF103C131
:100A30000FF104C110F105C111F106C112F107C196
:100A400013F108C114F109C115F10AC116F10BC166
:100A500017F134C135F111B839EF05F00101620E1B
:100A6000046F010E056F000E066F000E076F42EF58
:100A700005F00101A70E046F020E056F000E066F50
:100A8000000E076F5EC100F15FC101F160C102F1AC
:100A900061C103F12CEC29F003BF04D018BE02D0D1
:100AA00018A0108C11A05AEF05F010BA5AEF05F0FB
:100AB0000F80108A0CC100F10DC101F10EC102F1CD
:100AC0000FC103F110C104F111C105F112C106F10A
:100AD00013C107F114C108F115C109F116C10AF1DA
:100AE00017C10BF135C134F1FCEF0AF00392ABB240
:100AF000AB98AB88030103EE00F080517F0BE92631
:100B000004C0EFFF802B8151805D700BD8A48B82D5
:100B100000008051815D700BD8A48B9281518019A7
:100B2000D8B40790FCEF0AF0F2940101453FFCEFC6
:100B30000AF0462BFCEF0AF09E900101533FFCEFB8
:100B40000AF0542BFCEF0AF09E9211B821EF08F046
:100B5000040062A1ACEF05F08BB4B6EF05F010AC69
:100B6000B6EF05F08B84109CB7EF05F08B94077CF3
:100B700007ACD2EF05F0C274C2B4CCEF05F0C3CF1E
:100B8000B3F5C4CFB4F50501D890B433B333D890DE
:100B9000B433B333D3EF05F0C3CF55F1C4CF56F11F
:100BA000D3EF05F0C28207B440EF06F047C14BF126
:100BB00048C14CF149C14DF14AC14EF15EC162F1EB
:100BC0005FC163F160C164F161C165F196C1B6F1C5
:100BD00097C1B7F198C1B8F199C1B9F19AC1BAF109
:100BE0009BC1BBF19CC1BCF19DC1BDF19EC1BEF1D9
:100BF0009FC1BFF1A0C1C0F1A1C1C1F1A2C1C2F1A9
:100C0000A3C1C3F1A4C1C4F1A5C1C5F1A6C1C6F178
:100C1000A7C1C7F1A8C1C8F1A9C1C9F1AAC1CAF148
:100C2000ABC1CBF1ACC1CCF1ADC1CDF1AEC1CEF118
:100C3000AFC1CFF1B0C1D0F1B1C1D1F1B2C1D2F1E8
:100C4000B3C1D3F1B4C1D4F1B5C1D5F1B3C5B5F5D4
:100C5000B4C5B6F5B5C5B7F5B6C5B8F5010155517A
:100C60005B2756515C23E86A5D230E2E40EF06F0A9
:100C70005CC157F15DC158F15B6B5C6B5D6B078EBE
:100C80000201002FFCEF0AF03C0E006F1950E00B40
:100C9000E00AE866128817BE02D017B4108E00C1B1
:100CA0000CF101C10DF102C10EF103C10FF104C13C
:100CB00010F105C111F106C112F107C113F108C10C
:100CC00014F109C115F10AC116F10BC117F134C1B4
:100CD00035F105012F51000AD8B41AEF07F00501CC
:100CE0002F51010AD8B4A4EF06F005012F51020AD2
:100CF000D8B4E5EF06F005012F51030AD8B4E5EFAB
:100D000006F005012F51040AD8B4E5EF06F00501FD
:100D10002F51050AD8B4E5EF06F005012F51060A58
:100D2000D8B4E5EF06F005012F51070AD8B4E5EF76
:100D300006F005012F51320AD8B4A2EF06F02F6B4E
:100D40001AEF07F01AEF07F005015367AFEF06F04F
:100D50005467AFEF06F05567AFEF06F05667B3EF95
:100D600006F01AEF07F057C500F158C501F159C553
:100D700002F15AC503F10101010E046F000E056F67
:100D8000000E066F000E076F2CEC29F000C157F51E
:100D900001C158F502C159F503C15AF50067D8EFF2
:100DA00006F00167D8EF06F00267D8EF06F0036798
:100DB0001AEF07F053C557F554C558F555C559F501
:100DC00056C55AF50F881AEF07F005013067EBEFAB
:100DD00006F01AEF07F00FBE00EF07F010A005EFC6
:100DE00007F001014767FCEF06F04867FCEF06F0EB
:100DF0004967FCEF06F04A6700EF07F005EF07F0E0
:100E000007AE05EF07F017EF07F00501312F1AEFD6
:100E100007F03C0E316F302F1AEF07F00101000E82
:100E2000626FE00E636FA50E646F010E656F0501C2
:100E3000306B0F880501626B33B720EF07F06281DA
:100E40000CC100F10DC101F10EC102F10FC103F19E
:100E500010C104F111C105F112C106F113C107F16E
:100E600014C108F115C109F116C10AF117C10BF13E
:100E700035C134F100C10CF101C10DF102C10EF117
:100E800003C10FF104C110F105C111F106C112F146
:100E900007C113F108C114F109C115F10AC116F116
:100EA0000BC117F134C135F101018A675FEF07F01B
:100EB0008B675FEF07F08C675FEF07F08D6763EF7D
:100EC00007F093EF07F08EC100F18FC101F190C1DF
:100ED00002F191C103F10101010E046F000E056FD3
:100EE000000E066F000E076F2CEC29F000C18EF18A
:100EF00001C18FF102C190F103C191F1006788EF48
:100F000007F0016788EF07F0026788EF07F00367D3
:100F100093EF07F08AC18EF18BC18FF18CC190F1F4
:100F20008DC191F10F80D57ED5BE6DD0D6CF47F162
:100F3000D7CF48F145C149F1E86AE8CF4AF118BE78
:100F400002D018A0108C109047C100F148C101F1E7
:100F500049C102F14AC103F101010A0E046F000EFA
:100F6000056F000E066F000E076F2CEC29F003AF23
:100F70001080010154A7C9EF07F00F9A0F9C0F9E34
:100F80000101000E5E6F600E5F6F3D0E606F080E18
:100F9000616F010147BFD9EF07F04867D9EF07F04C
:100FA0004967D9EF07F04A67D9EF07F0F288FEEFFB
:100FB00007F0F2985E6B5F6B606B616B966B976B83
:100FC000986B996B9A6B9B6B9C6B9D6B9E6B9F6BED
:100FD000A06BA16BA26BA36BA46BA56BA66BA76B9D
:100FE000A86BA96BAA6BAB6BAC6BAD6BAE6BAF6B4D
:100FF000B06BB16BB26BB36BB46BB56BD76AD66ABF
:101000000101456B466B0CC100F10DC101F10EC130
:1010100002F10FC103F110C104F111C105F112C1B8
:1010200006F113C107F114C108F115C109F116C188
:101030000AF117C10BF135C134F1FCEF0AF0FCEFF6
:101040000AF00201002F65EF0AF0D59ED6CF47F1D6
:10105000D7CF48F145C149F1E86AE8CF4AF1D76AEC
:10106000D66A0101456B466BD58E1950E00BE00A3C
:10107000E866128817BE02D017B4108E16AE1B8C0D
:1010800000C10CF101C10DF102C10EF103C10FF15C
:1010900004C110F105C111F106C112F107C113F12C
:1010A00008C114F109C115F10AC116F10BC117F1FC
:1010B00034C135F10FA0109A11B86AEF08F00101A0
:1010C000620E046F010E056F000E066F000E076FB3
:1010D00073EF08F00101A70E046F020E056F000EFA
:1010E000066F000E076F47C100F148C101F149C109
:1010F00002F14AC103F12CEC29F003BF86EF08F09E
:1011000018BE02D018A0108C11B00F800CC100F1D5
:101110000DC101F10EC102F10FC103F110C104F1C3
:1011200011C105F112C106F113C107F114C108F193
:1011300015C109F116C10AF117C10BF135C134F11E
:1011400002013C0E006F00C10CF101C10DF102C1A2
:101150000EF103C10FF104C110F105C111F106C177
:1011600012F107C113F108C114F109C115F10AC147
:1011700016F10BC117F134C135F105012F51000AE9
:10118000D8B46EEF09F005012F51010AD8B4F8EF79
:1011900008F005012F51020AD8B439EF09F0050112
:1011A0002F51030AD8B439EF09F005012F51040A71
:1011B000D8B439EF09F005012F51050AD8B439EF39
:1011C00009F005012F51060AD8B439EF09F00501DD
:1011D0002F51070AD8B439EF09F005012F51320A0F
:1011E000D8B4F6EF08F02F6B6EEF09F06EEF09F050
:1011F0000501536703EF09F0546703EF09F05567E2
:1012000003EF09F0566707EF09F06EEF09F057C5D5
:1012100000F158C501F159C502F15AC503F10101A8
:10122000010E046F000E056F000E066F000E076FB3
:101230002CEC29F000C157F501C158F502C159F550
:1012400003C15AF500672CEF09F001672CEF09F094
:1012500002672CEF09F003676EEF09F053C557F5ED
:1012600054C558F555C559F556C55AF50F886EEF52
:1012700009F0050130673FEF09F06EEF09F00FBE8E
:1012800054EF09F010A059EF09F00101476750EF42
:1012900009F0486750EF09F0496750EF09F04A67D5
:1012A00054EF09F059EF09F007AE59EF09F06BEF71
:1012B00009F00501312F6EEF09F03C0E316F302F30
:1012C0006EEF09F00101000E626FE00E636FA50E74
:1012D000646F010E656F0501306B0F880501626B4D
:1012E00033B774EF09F062810CC100F10DC101F157
:1012F0000EC102F10FC103F110C104F111C105F1DA
:1013000012C106F113C107F114C108F115C109F1A9
:1013100016C10AF117C10BF135C134F100C10CF14E
:1013200001C10DF102C10EF103C10FF104C110F1B1
:1013300005C111F106C112F107C113F108C114F181
:1013400009C115F10AC116F10BC117F134C135F10C
:1013500001018A67B3EF09F08B67B3EF09F08C677F
:10136000B3EF09F08D67B7EF09F0E7EF09F08EC131
:1013700000F18FC101F190C102F191C103F10101AE
:10138000010E046F000E056F000E066F000E076F52
:101390002CEC29F000C18EF101C18FF102C190F156
:1013A00003C191F10067DCEF09F00167DCEF09F0A0
:1013B0000267DCEF09F00367E7EF09F08AC18EF1FD
:1013C0008BC18FF18CC190F18DC191F10F80109084
:1013D00047C100F148C101F149C102F14AC103F11D
:1013E00001010A0E046F000E056F000E066F000E5D
:1013F000076F2CEC29F003AF1080010154A70DEF0B
:101400000AF00F9A0F9C0F9E0101000E5E6F600E96
:101410005F6F3D0E606F080E616F47C100F148C1FC
:1014200001F149C102F14AC103F10101140E046F37
:10143000050E056F000E066F000E076F2CEC29F0ED
:1014400003AF26EF0AF0F2884BEF0AF0F2985E6BDA
:101450005F6B606B616B966B976B986B996B9A6B1C
:101460009B6B9C6B9D6B9E6B9F6BA06BA16BA26B30
:10147000A36BA46BA56BA66BA76BA86BA96BAA6BE0
:10148000AB6BAC6BAD6BAE6BAF6BB06BB16BB26B90
:10149000B36BB46BB56B0CC100F10DC101F10EC1A2
:1014A00002F10FC103F110C104F111C105F112C124
:1014B00006F113C107F114C108F115C109F116C1F4
:1014C0000AF117C10BF135C134F104008BB470EF90
:1014D0000AF010AC70EF0AF08B84109C71EF0AF0E8
:1014E0008B94077C07AC8CEF0AF0C274C2B486EF11
:1014F0000AF0C3CFB3F5C4CFB4F50501D890B43327
:10150000B333D890B433B3338DEF0AF0C3CF55F172
:10151000C4CF56F18DEF0AF0C28207B4FAEF0AF099
:1015200047C14BF148C14CF149C14DF14AC14EF19F
:101530005EC162F15FC163F160C164F161C165F1D7
:1015400096C1B6F197C1B7F198C1B8F199C1B9F197
:101550009AC1BAF19BC1BBF19CC1BCF19DC1BDF167
:101560009EC1BEF19FC1BFF1A0C1C0F1A1C1C1F137
:10157000A2C1C2F1A3C1C3F1A4C1C4F1A5C1C5F107
:10158000A6C1C6F1A7C1C7F1A8C1C8F1A9C1C9F1D7
:10159000AAC1CAF1ABC1CBF1ACC1CCF1ADC1CDF1A7
:1015A000AEC1CEF1AFC1CFF1B0C1D0F1B1C1D1F177
:1015B000B2C1D2F1B3C1D3F1B4C1D4F1B5C1D5F147
:1015C000B3C5B5F5B4C5B6F5B5C5B7F5B6C5B8F587
:1015D000010155515B2756515C23E86A5D230E2EAD
:1015E000FAEF0AF05CC157F15DC158F15B6B5C6BBF
:1015F0005D6B078EFCEF0AF002C0E0FF005001C0F7
:10160000D8FF1000A6B202EF0BF00CC0A9FF0BC070
:10161000A8FFA69EA69CA684F29E550EA76EAA0EB3
:10162000A76EA682F28EA694A6B214EF0BF00C2A37
:101630001200A96EA69EA69CA680A8500C2A120095
:1016400004012C0E826F5BEC0EF027EC2AF00C509C
:1016500019EC0BF0E8CF00F10C5019EC0BF0E8CFCF
:1016600001F101AF39EF0BF00101FF0E026FFF0E28
:10167000036FCAEC29F0296745EF0BF00401200E37
:10168000826F5BEC0EF04AEF0BF004012D0E826FBF
:101690005BEC0EF0F4EC27F01200076A0F6A106A98
:1016A000116A126A0F010D0EC16E860EC06E030E16
:1016B000C26E0F01680E896E130E926E080E8A6E4E
:1016C000F30E936E8B6A900E946EC80E19EC0BF0AD
:1016D000E8CFE8FF1098E8A0108810A805D00E0EFB
:1016E000216E8E0E226E04D00F0E216E8F0E226E92
:1016F000A6EC2AF0F18EF19EFC0E19EC0BF0E8CF6F
:101700000BF00BA011800BA211820BA411840BA86B
:101710001188C90E19EC0BF0E8CF16F0CA0E19ECBF
:101720000BF0E8CF17F0CB0E19EC0BF0E8CF18F068
:10173000CC0E19EC0BF0E8CF19F01B6A1C6A0E6A8C
:1017400001015B6B5C6B5D6B576B586BF29A01012F
:10175000476B486B496B4A6B4B6B4C6B4D6B4E6BDD
:101760004F6B506B516B526B456B466BD76AD66AA9
:101770000F01280ED56EF28A9D90B00ECD6E01013C
:101780005E6B5F6B606B616B626B636B646B656BF5
:10179000666B676B686B696B536B546BCF6ACE6A11
:1017A0000F9A0F9C0F9E9D80760ECA6E9D8202013D
:1017B0003C0E006FCC6A160E19EC0BF0E8CF00F16E
:1017C000170E19EC0BF0E8CF01F1180E19EC0BF025
:1017D000E8CF02F1190E19EC0BF0E8CF03F101018B
:1017E00003AF0DEF0CF027EC2AF0160E0C6E00C1C3
:1017F0000BF002EC0BF0170E0C6E01C10BF002ECBB
:101800000BF0180E0C6E02C10BF002EC0BF0190E6F
:101810000C6E03C10BF002EC0BF000C18AF101C1A8
:101820008BF102C18CF103C18DF100C18EF101C1B8
:101830008FF102C190F103C191F11A0E19EC0BF076
:10184000E8CF00F11B0E19EC0BF0E8CF01F11C0EF4
:1018500019EC0BF0E8CF02F11D0E19EC0BF0E8CFFC
:1018600003F1010103AF63EF0CF027EC2AF01A0E2D
:101870000C6E00C10BF002EC0BF01B0E0C6E01C1E4
:101880000BF002EC0BF01C0E0C6E02C10BF002EC24
:101890000BF01D0E0C6E03C10BF002EC0BF01A0ED8
:1018A00019EC0BF0E8CF00F11B0E19EC0BF0E8CFB0
:1018B00001F11C0E19EC0BF0E8CF02F11D0E19EC32
:1018C0000BF0E8CF03F100C192F101C193F102C125
:1018D00094F103C195F1240EAC6E900EAB6E240E04
:1018E000AC6E080EB86E000EB06E1F0EAF6E040127
:1018F000806B816B0F01900EAB6E0F019D8A03010F
:10190000806B816BC26B8B922EEC2FF02EEC2FF044
:101910008AEC30F00DEC2DF0200E19EC0BF0E8CF36
:101920002FF505012F51FF0AD8A49EEF0CF02F6B65
:10193000200E0C6E2FC50BF002EC0BF00501010E12
:10194000306F3C0E316F250E19EC0BF0E8CF00F133
:10195000260E19EC0BF0E8CF01F1270E19EC0BF075
:10196000E8CF02F1280E19EC0BF0E8CF03F10101EA
:1019700003AFD5EF0CF027EC2AF0250E0C6E00C15A
:101980000BF002EC0BF0260E0C6E01C10BF002EC1A
:101990000BF0270E0C6E02C10BF002EC0BF0280EC0
:1019A0000C6E03C10BF002EC0BF000C153F501C14A
:1019B00054F502C155F503C156F500C157F501C1F3
:1019C00058F502C159F503C15AF5290E19EC0BF06F
:1019D000E8CF5BF505015C515B5DD8A05BC55CF5AC
:1019E00005012F51020A0EE181B802EF0DF0050149
:1019F0005C2FFFEF0CF05BC55CF502EF0DF081BAD8
:101A0000C9EF30F0210E19EC0BF0E8CF00F1220EF7
:101A100019EC0BF0E8CF01F1230E19EC0BF0E8CF35
:101A200002F1240E19EC0BF0E8CF03F1010103AF32
:101A300048EF0DF027EC2AF0210E0C6E00C10BF0E0
:101A400002EC0BF0220E0C6E01C10BF002EC0BF05D
:101A5000230E0C6E02C10BF002EC0BF0240E0C6E88
:101A600003C10BF002EC0BF0210E19EC0BF0E8CFE8
:101A700000F1220E19EC0BF0E8CF01F1230E19EC66
:101A80000BF0E8CF02F1240E19EC0BF0E8CF03F1D4
:101A900000C15DF501C15EF502C15FF503C160F5EE
:101AA00055EC2CF057EC2BF0AFEC2AF005012F5140
:101AB000030A12E005012F51040A1DE005012F5110
:101AC000050A24E005012F51060A32E005012F51D5
:101AD000070A38E0ABEF0DF0ACC500F101010F0EC5
:101AE000001701010051000A36E001010051050A0A
:101AF00032E0A8EF0DF0ACC500F101010F0E0017A8
:101B000001010051000A27E0A8EF0DF00501AC51DA
:101B1000000A21E00501AC51150A1DE00501AC5198
:101B2000300A19E00501AC51450A15E0A8EF0DF0A7
:101B30000501AC51000A0FE00501AC51300A0BE081
:101B4000A8EF0DF00501AC51000A05E0A8EF0DF07B
:101B500081BAC9EF30F007900001F28EF28C07B025
:101B600078EF26F00FB014EF20F010BE14EF20F045
:101B700012B814EF20F00FB8B3EF19F00301805141
:101B800081197F0BD8B478EF26F013EE00F0815165
:101B90007F0BE126812BE7CFE8FFE00BD8B478EF8D
:101BA00026F023EE82F0C2513F0BD926E7CFDFFFAC
:101BB000C22BDF50780AD8A478EF26F007808EC1B8
:101BC00000F18FC101F190C102F191C103F1010156
:101BD000040E046F000E056F000E066F000E076FF7
:101BE0002CEC29F000AFFEEF0DF00101030E8E6F1B
:101BF000000E8F6F000E906F000E916F03018251E7
:101C0000720AD8B4FBEF1FF08251520AD8B4FBEF2E
:101C10001FF08251750AD8B4FBEF1FF08251630A9E
:101C2000D8B432EF23F08251690AD8B4AAEF1CF07D
:101C300082517A0AD8B4BDEF1DF08251490AD8B456
:101C400049EF1CF08251500AD8B467EF1BF0825163
:101C5000700AD8B4AAEF1BF08251540AD8B4D5EF59
:101C60001BF08251740AD8B41BEF1CF08251410A58
:101C7000D8B46FEF0EF082516D0AD8B479EF12F03C
:101C800082514D0AD8B492EF12F08251730AD8B43F
:101C90002BEF1FF08251530AD8B490EF1FF08251FE
:101CA0004C0AD8B421EF13F08251590AD8B4CAEFC4
:101CB00011F069EF23F0040114EE00F080517F0B66
:101CC000E12682C4E7FF802B120004010D0E826F13
:101CD0005BEC0EF00A0E826F5BEC0EF0120004015A
:101CE000410E826F5BEC0EF003018351310AD8B4D0
:101CF000EAEF10F003018351320AD8B41AEF10F062
:101D000003018351330AD8B4A3EF0FF003018351C9
:101D1000340AD8B493EF0EF004013F0E826F5BECEF
:101D20000EF067EF23F0CC0E19EC0BF0E8CF0BF0C0
:101D300004012C0E826F5BEC0EF003018451310A1A
:101D4000D8B4B7EF0EF003018451300AD8B4B9EF1C
:101D50000EF0030184514D0AD8B4C3EF0EF0030115
:101D60008451540AD8B4CAEF0EF0E1EF0EF08A8421
:101D700001D08A940BAE04D00BAC02D00BBA21D0A8
:101D8000E00E0B1218D01F0E0B168539E844E00B3D
:101D90000B1211D0E00E0B1668EC2AF085C332F15D
:101DA00086C333F10101296B75EC2AF0ECEC29F0C4
:101DB00000511F0B0B12CC0E0C6E0BC00BF002EC83
:101DC0000BF00401340E826F5BEC0EF004012C0E5C
:101DD000826F5BEC0EF0CC0E19EC0BF0E8CF19F033
:101DE0008AB406D00401300E826F5BEC0EF005D091
:101DF0000401310E826F5BEC0EF004012C0E826F39
:101E00005BEC0EF01938E840070BE8CF82F40401D0
:101E1000300E82275BEC0EF004012C0E826F5BEC1F
:101E20000EF027EC2AF019501F0BE8CF00F1CAEC96
:101E300029F032C182F40401300E82275BEC0EF0EF
:101E400033C182F40401300E82275BEC0EF00401F2
:101E50002C0E826F5BEC0EF027EC2AF02CC000F108
:101E600000AF0BD0FF0E016FFF0E026FFF0E036F6E
:101E700004012D0E826F5BEC0EF0CAEC29F031C12B
:101E800082F40401300E82275BEC0EF032C182F442
:101E90000401300E82275BEC0EF033C182F40401A2
:101EA000300E82275BEC0EF004012C0E826F5BEC8F
:101EB0000EF027EC2AF02BC000F1CAEC29F031C15A
:101EC00082F40401300E82275BEC0EF032C182F402
:101ED0000401300E82275BEC0EF033C182F4040162
:101EE000300E82275BEC0EF004012C0E826F5BEC4F
:101EF0000EF027EC2AF02DC000F100AF0BD0FF0E42
:101F0000016FFF0E026FFF0E036F04012D0E826F33
:101F10005BEC0EF0CAEC29F031C182F40401300E02
:101F200082275BEC0EF032C182F40401300E82276E
:101F30005BEC0EF033C182F40401300E82275BECBF
:101F40000EF067EF23F0CB0E19EC0BF0E8CF0BF09F
:101F500004012C0E826F5BEC0EF003018451450AE4
:101F6000D8B4C7EF0FF003018451440AD8B4CAEFC4
:101F70000FF003018451300AD8B4CDEF0FF0030104
:101F80008451310AD8B4D1EF0FF0DCEF0FF00B9E83
:101F9000D6EF0FF00B8ED6EF0FF0FC0E0B16D6EF30
:101FA0000FF0FC0E0B160B80D6EF0FF0CB0E0C6E65
:101FB0000BC00BF002EC0BF00401330E826F5BECF4
:101FC0000EF004012C0E826F5BEC0EF0CB0E19ECC0
:101FD0000BF0E8CF18F018BEF5EF0FF00401450E36
:101FE000826F5BEC0EF0FAEF0FF00401440E826F8B
:101FF0005BEC0EF004012C0E826F5BEC0EF0040122
:10200000300E826F5BEC0EF004012C0E826F5BECE5
:102010000EF018B013EF10F00401300E826F5BEC7D
:102020000EF018EF10F00401310E826F5BEC0EF031
:1020300067EF23F0CA0E19EC0BF0E8CF0BF00401A8
:102040002C0E826F5BEC0EF003018451450AD8B46C
:1020500056EF10F003018451440AD8B459EF10F040
:10206000030184514D0AD8B462EF10F0030184518A
:10207000410AD8B45CEF10F003018451460AD8B489
:102080005FEF10F003018451560AD8B46AEF10F0E4
:1020900003018451500AD8B475EF10F00301845144
:1020A000520AD8B478EF10F081EF10F00B9E7BEF5E
:1020B00010F00B8E7BEF10F00B9C7BEF10F00B8C75
:1020C0007BEF10F0FC0E0B1685C3E8FF030B0B1221
:1020D0007BEF10F0C70E0B1685C3E8FF070BE84631
:1020E000E846E8460B127BEF10F00B847BEF10F014
:1020F0000B947BEF10F0CA0E0C6E0BC00BF002ECD1
:102100000BF0CA0E19EC0BF0E8CF17F00401320EF9
:10211000826F5BEC0EF004012C0E826F5BEC0EF014
:1021200017BE9AEF10F00401450E826F5BEC0EF0C3
:102130009FEF10F00401440E826F5BEC0EF004017F
:102140002C0E826F5BEC0EF017C0E8FF030BE8CF9C
:1021500082F40401300E82275BEC0EF004012C0E99
:10216000826F5BEC0EF017BCBDEF10F00401410E66
:10217000826F5BEC0EF0C2EF10F00401460E826F2E
:102180005BEC0EF004012C0E826F5BEC0EF017C0BE
:10219000E8FF380BE842E842E842E8CF82F4040165
:1021A000300E82275BEC0EF004012C0E826F5BEC8C
:1021B0000EF017B4E3EF10F00401520E826F5BECE7
:1021C0000EF0E8EF10F00401500E826F5BEC0EF0A1
:1021D00067EF23F0C90E19EC0BF0E8CF0BF0040108
:1021E0002C0E826F5BEC0EF003018451450AD8B4CB
:1021F00008EF11F003018451440AD8B40BEF11F039
:10220000030184514D0AD8B40EEF11F01CEF11F008
:102210000B9E16EF11F00B8E16EF11F0F80E0B1649
:1022200085C3E8FF070B0B1216EF11F0C90E0C6EF9
:102230000BC00BF002EC0BF00401310E826F5BEC73
:102240000EF004012C0E826F5BEC0EF0C90E19EC3F
:102250000BF0E8CF16F016BE06D00401450E826FD3
:102260005BEC0EF005D00401440E826F5BEC0EF0C7
:1022700004012C0E826F5BEC0EF016C0E8FF070B1A
:10228000E8CF82F40401300E82275BEC0EF00401EB
:102290002C0E826F5BEC0EF0078027EC2AF027C033
:1022A000E8FF003B00430043030BCAEC29F033C1B5
:1022B00082F40401300E82275BEC0EF004012C0E38
:1022C000826F5BEC0EF027EC2AF027C001F1019F32
:1022D000019D28C000F10101CAEC29F02FC182F450
:1022E0000401300E82275BEC0EF030C182F4040151
:1022F000300E82275BEC0EF031C182F40401300E07
:1023000082275BEC0EF032C182F40401300E82278A
:102310005BEC0EF033C182F40401300E82275BECDB
:102320000EF004012C0E826F5BEC0EF027EC2AF00D
:1023300029C001F12AC000F1D89001330033D890B0
:10234000013300330101CAEC29F02FC182F40401EA
:10235000300E82275BEC0EF030C182F40401300EA7
:1023600082275BEC0EF031C182F40401300E82272B
:102370005BEC0EF032C182F40401300E82275BEC7C
:102380000EF033C182F40401300E82275BEC0EF0B4
:1023900067EF23F0FC0E19EC0BF0E8CF0BF0030114
:1023A0008351520AD8B401EF12F003018351720A2B
:1023B000D8B404EF12F003018351500AD8B407EFE8
:1023C00012F003018351700AD8B40AEF12F003012E
:1023D0008351550AD8B40DEF12F003018351750AE9
:1023E000D8B410EF12F003018351430AD8B419EFA7
:1023F00012F003018351630AD8B41CEF12F025EFE9
:1024000012F00B901FEF12F00B801FEF12F00B92E7
:102410001FEF12F00B821FEF12F00B941FEF12F060
:102420000B841FEF12F00B961FEF12F00B861FEFBD
:1024300012F00B981FEF12F00B881FEF12F0FC0E3A
:102440000C6E0BC00BF002EC0BF00401590E826F06
:102450005BEC0EF01190119211941198FC0E19EC96
:102460000BF0E8CF0BF00BA011800BA211820BA494
:1024700011840BA8118811A045EF12F00401520E2F
:10248000826F5BEC0EF04AEF12F00401720E826F65
:102490005BEC0EF011A854EF12F00401430E826FB2
:1024A0005BEC0EF059EF12F00401630E826F5BECEF
:1024B0000EF011A263EF12F00401500E826F5BEC7C
:1024C0000EF068EF12F00401700E826F5BEC0EF0FC
:1024D00011A472EF12F00401550E826F5BEC0EF046
:1024E00077EF12F00401750E826F5BEC0EF067EF70
:1024F00023F004016D0E826F5BEC0EF0030183513B
:10250000300AD8B4D1EF12F003018351310AD8B4A4
:10251000E4EF12F003018351320AD8B4F7EF12F05E
:1025200069EF23F004014D0E826F5BEC0EF068EC56
:102530002AF084C331F185C332F186C333F101013E
:10254000296B75EC2AF0ECEC29F003018351300A79
:10255000D8B4B9EF12F003018351310AD8B4C1EFF6
:1025600012F003018351320AD8B4C9EF12F069EFB7
:1025700023F0FD0E0C6E00C10BF002EC0BF0D1EF5E
:1025800012F0FE0E0C6E00C10BF002EC0BF0E4EF4B
:1025900012F0FF0E0C6E00C10BF002EC0BF0F7EF27
:1025A00012F00401300E826F5BEC0EF004012C0E71
:1025B000826F5BEC0EF027EC2AF0FD0E19EC0BF0AD
:1025C000E8CF00F108EF13F00401310E826F5BECED
:1025D0000EF004012C0E826F5BEC0EF027EC2AF05B
:1025E000FE0E19EC0BF0E8CF00F108EF13F0040138
:1025F000320E826F5BEC0EF027EC2AF004012C0EF9
:10260000826F5BEC0EF0FF0E19EC0BF0E8CF00F1DF
:10261000CAEC29F031C182F40401300E82275BEC50
:102620000EF032C182F40401300E82275BEC0EF012
:1026300033C182F40401300E82275BEC0EF067EFA9
:1026400023F003018351300AD8B48CEF16F0030154
:102650008351310AD8B4B9EF17F003018351320A1C
:10266000D8B427EF18F003018351330AD8B437EFF9
:1026700018F003018351340AD8B447EF18F003016E
:102680008351350AD8B4B8EF19F003018351360AE3
:10269000D8B4E6EF19F003018351370AD8B4EEEF4E
:1026A00015F003018351460AD8B40CEF19F0030169
:1026B00083514D0AD8B467EF14F0030183516D0ABA
:1026C000D8B481EF14F0030183515A0AD8B433EF20
:1026D00017F003018351490AD8B4E6EF1AF0030159
:1026E0008351500AD8B418EF1AF003018351540AE9
:1026F000D8B491EF1AF003018351630AD8B4A1EF63
:1027000014F003018351430AD8B499EF15F0030183
:102710008351730AD8B49FEF14F003018351610A07
:10272000D8B4B4EF13F003018351650AD8B4DCEFD9
:1027300016F003018351450AD8B4EAEF16F00301FD
:102740008351620AD8B4F8EF16F003018351420AAC
:10275000D8B406EF17F003018351760AD8B414EF0A
:1027600017F0D8A469EF23F004014C0E826F5BECE4
:102770000EF00401610E826F5BEC0EF057EC2BF053
:1027800004012C0E826F5BEC0EF027EC2AF0ABC537
:1027900000F10101CAEC29F031C182F40401300ECC
:1027A00082275BEC0EF032C182F40401300E8227E6
:1027B0005BEC0EF033C182F40401300E82275BEC37
:1027C0000EF004012C0E826F5BEC0EF027EC2AF069
:1027D000ACC500F10101CAEC29F031C182F4040159
:1027E000300E82275BEC0EF032C182F40401300E11
:1027F00082275BEC0EF033C182F40401300E822795
:102800005BEC0EF004012C0E826F5BEC0EF027ECFB
:102810002AF0ADC500F10101CAEC29F031C182F402
:102820000401300E82275BEC0EF032C182F4040109
:10283000300E82275BEC0EF033C182F40401300EBF
:1028400082275BEC0EF004012C0E826F5BEC0EF025
:1028500027EC2AF0AEC500F10101CAEC29F031C124
:1028600082F40401300E82275BEC0EF032C182F458
:102870000401300E82275BEC0EF033C182F40401B8
:10288000300E82275BEC0EF004012C0E826F5BECA5
:102890000EF027EC2AF0B2C500F10101CAEC29F0D4
:1028A00031C182F40401300E82275BEC0EF032C19C
:1028B00082F40401300E82275BEC0EF033C182F407
:1028C0000401300E82275BEC0EF014EF1AF068EC76
:1028D0002AF084C333F175EC2AF0ECEC29F0200ED9
:1028E0000C6E00C10BF002EC0BF000C12FF50501DE
:1028F0002F51000A06E005012F51010A02E0F1EC18
:102900002BF004014C0E826F5BEC0EF004014D0EB7
:10291000826F5BEC0EF004012C0E826F5BEC0EF00C
:1029200027EC2AF02FC500F1CAEC29F033C182F45C
:102930000401300E82275BEC0EF014EF1AF0C9EFA1
:1029400030F004014C0E826F5BEC0EF00401630E5C
:10295000826F5BEC0EF0AFEC2AF004012C0E826F5C
:102960005BEC0EF0B6EC14F014EF1AF027EC2AF042
:10297000B1C500F10101003B0F0E0017CAEC29F0B0
:1029800033C182F40401300E82275BEC0EF0B1C536
:1029900000F101010F0E01010017CAEC29F033C14B
:1029A00082F40401300E82275BEC0EF004012D0E40
:1029B000826F5BEC0EF0B0C500F10101003B0F0E21
:1029C0000017CAEC29F033C182F40401300E8227CB
:1029D0005BEC0EF0B0C500F101010F0E0101001714
:1029E000CAEC29F033C182F40401300E82275BEC7B
:1029F0000EF004012D0E826F5BEC0EF0AFC500F1FE
:102A00000101003B0F0E0017CAEC29F033C182F41C
:102A10000401300E82275BEC0EF0AFC500F101011E
:102A20000F0E01010017CAEC29F033C182F4040132
:102A3000300E82275BEC0EF00401200E826F5BECFF
:102A40000EF0AEC500F10F0E01010017CAEC29F01F
:102A500033C182F40401300E82275BEC0EF00401D6
:102A6000200E826F5BEC0EF0ADC500F1010101019B
:102A7000003B0F0E0017CAEC29F033C182F40401A9
:102A8000300E82275BEC0EF0ADC500F101010F0E98
:102A900001010017CAEC29F033C182F40401300EA1
:102AA00082275BEC0EF004013A0E826F5BEC0EF0B5
:102AB000ACC500F10101003B0F0E0017CAEC29F074
:102AC00033C182F40401300E82275BEC0EF0ACC5FA
:102AD00000F101010F0E01010017CAEC29F033C10A
:102AE00082F40401300E82275BEC0EF004013A0EF2
:102AF000826F5BEC0EF0ABC500F10101003B0F0EE5
:102B00000017CAEC29F033C182F40401300E822789
:102B10005BEC0EF0ABC500F101010F0E0017CAEC23
:102B200029F033C182F40401300E82275BEC0EF0F1
:102B3000120084C3E8FF0F0BE83AE8CFB1F585C374
:102B4000E8FF0F0B0501B11387C3E8FF0F0BE83A4D
:102B5000E8CFB0F588C3E8FF0F0B0501B0138AC3B7
:102B6000E8FF0F0BE83AE8CFAFF58BC3E8FF0F0B98
:102B70000501AF138DC3E8FF0F0BE8CFAEF58FC390
:102B8000E8FF0F0BE83AE8CFADF590C3E8FF0F0B75
:102B90000501AD1392C3E8FF0F0BE83AE8CFACF59F
:102BA00093C3E8FF0F0B0501AC1395C3E8FF0F0BB0
:102BB000E83AE8CFABF596C3E8FF0F0B0501AB137E
:102BC0000AEC2BF004014C0E826F5BEC0EF004015A
:102BD000430E826F5BEC0EF0ABEF14F00784040140
:102BE0004C0E826F5BEC0EF00401370E826F5BECD3
:102BF0000EF004012C0E826F5BEC0EF005012E51DD
:102C0000130A06E005012E51170A0DE089EF16F0B0
:102C10000101000E006F000E016F100E026F000E1A
:102C2000036F1CEF16F00101000E006F000E016F24
:102C3000000E026F010E036FCAEC29F02AC182F464
:102C40000401300E82275BEC0EF02BC182F40401EC
:102C5000300E82275BEC0EF02CC182F40401300EA2
:102C600082275BEC0EF02DC182F40401300E822726
:102C70005BEC0EF02EC182F40401300E82275BEC77
:102C80000EF02FC182F40401300E82275BEC0EF0AF
:102C900030C182F40401300E82275BEC0EF031C1AA
:102CA00082F40401300E82275BEC0EF032C182F414
:102CB0000401300E82275BEC0EF033C182F4040174
:102CC000300E82275BEC0EF004012C0E826F5BEC61
:102CD0000EF00101100E006F000E016F000E026F6A
:102CE000000E036FCAEC29F031C182F40401300EEA
:102CF00082275BEC0EF032C182F40401300E822791
:102D00005BEC0EF033C182F40401300E82275BECE1
:102D10000EF0079414EF1AF007848AEC30F027ECD9
:102D20002AF02DC500F1CAEC29F004014C0E826F87
:102D30005BEC0EF00401300E826F5BEC0EF00401D0
:102D40002C0E826F5BEC0EF031C182F40401300E68
:102D500082275BEC0EF032C182F40401300E822730
:102D60005BEC0EF033C182F40401300E82275BEC81
:102D70000EF004012C0E826F5BEC0EF027EC2AF0B3
:102D80002EC500F1CAEC29F031C182F40401300EE5
:102D900082275BEC0EF032C182F40401300E8227F0
:102DA0005BEC0EF033C182F40401300E82275BEC41
:102DB0000EF0079414EF1AF004014C0E826F5BECD6
:102DC0000EF00401650E826F5BEC0EF0B1EC2CF09E
:102DD00014EF1AF004014C0E826F5BEC0EF004014C
:102DE000450E826F5BEC0EF0C8EC2CF014EF1AF07D
:102DF00004014C0E826F5BEC0EF00401620E826FD8
:102E00005BEC0EF0F6EC2CF014EF1AF004014C0E13
:102E1000826F5BEC0EF00401420E826F5BEC0EF0F1
:102E2000DFEC2CF014EF1AF004014C0E826F5BEC17
:102E30000EF00401760E826F5BEC0EF004012C0E96
:102E4000826F5BEC0EF010A807D00401310E826F88
:102E50005BEC0EF014EF1AF00401300E826F5BECA5
:102E60000EF014EF1AF004014C0E826F5BEC0EF0C2
:102E700004015A0E826F5BEC0EF004012C0E826F7F
:102E80005BEC0EF08AEC30F027EC2AF005012E51B5
:102E9000130A06E005012E51170A0DE064EF17F042
:102EA0000101000E006F000E016F100E026F000E88
:102EB000036F64EF17F00101000E006F000E016F49
:102EC000000E026F010E036F0101100E046F000E61
:102ED000056F000E066F000E076F5DEC29F0CAEC5F
:102EE00029F02AC182F40401300E82275BEC0EF037
:102EF0002BC182F40401300E82275BEC0EF02CC152
:102F000082F40401300E82275BEC0EF02DC182F4B6
:102F10000401300E82275BEC0EF02EC182F4040116
:102F2000300E82275BEC0EF02FC182F40401300ECC
:102F300082275BEC0EF030C182F40401300E822750
:102F40005BEC0EF031C182F40401300E82275BECA1
:102F50000EF032C182F40401300E82275BEC0EF0D9
:102F600033C182F40401300E82275BEC0EF014EFC3
:102F70001AF0078404014C0E826F5BEC0EF0040122
:102F8000310E826F5BEC0EF004012C0E826F5BEC55
:102F90000EF025C500F126C501F127C502F128C5AF
:102FA00003F10101100E046F000E056F000E066F95
:102FB000000E076F5DEC29F0CAEC29F02AC182F4FB
:102FC0000401300E82275BEC0EF02BC182F4040169
:102FD000300E82275BEC0EF02CC182F40401300E1F
:102FE00082275BEC0EF02DC182F40401300E8227A3
:102FF0005BEC0EF02EC182F40401300E82275BECF4
:103000000EF02FC182F40401300E82275BEC0EF02B
:1030100030C182F40401300E82275BEC0EF031C126
:1030200082F40401300E82275BEC0EF032C182F490
:103030000401300E82275BEC0EF033C182F40401F0
:10304000300E82275BEC0EF0079414EF1AF0078421
:1030500004014C0E826F5BEC0EF00401320E826FA5
:103060005BEC0EF0E4EC2EF0079414EF1AF00784FA
:1030700004014C0E826F5BEC0EF00401330E826F84
:103080005BEC0EF041EC2FF00794C4EF17F00784CF
:1030900004014C0E826F5BEC0EF00401340E826F63
:1030A0005BEC0EF004012C0E826F5BEC0EF068EC12
:1030B0002AF084C32AF185C32BF186C32CF187C380
:1030C0002DF188C32EF189C32FF18AC330F18BC350
:1030D00031F18CC332F18DC333F10101296B75ECF1
:1030E0002AF0ECEC29F0100E046F000E056F000EB4
:1030F000066F000E076F3DEC29F000C121F501C1FC
:1031000022F502C123F503C124F53DEC30F034C5AE
:10311000ABF535C5ACF536C5ADF537C5AEF538C53B
:10312000AFF539C5B0F53AC5B1F5B6EC14F0040108
:103130002C0E826F5BEC0EF03BC500F13CC501F13B
:103140003DC502F13EC503F10101000E046F000E02
:10315000056F010E066F000E076F5DEC29F0CAECDB
:1031600029F02967B6EF18F0BBEF18F004012D0E17
:10317000826F5BEC0EF030C182F40401300E8227C6
:103180005BEC0EF031C182F40401300E82275BEC5F
:103190000EF004012E0E826F5BEC0EF032C182F451
:1031A0000401300E82275BEC0EF033C182F404017F
:1031B000300E82275BEC0EF004012C0E826F5BEC6C
:1031C0000EF027EC2AF03FC500F140C501F193EC69
:1031D00024F004012C0E826F5BEC0EF027EC2AF039
:1031E00041C500F1CAEC29F031C182F40401300E6E
:1031F00082275BEC0EF032C182F40401300E82278C
:103200005BEC0EF033C182F40401300E82275BECDC
:103210000EF0079414EF1AF068EC2AF085C32AF137
:1032200086C32BF187C32CF188C32DF189C32EF1FE
:103230008AC32FF18BC330F18CC331F18DC332F1CE
:103240008EC333F10101296B75EC2AF0ECEC29F007
:103250000101010E046F000E056F000E066F000ED7
:10326000076F2CEC29F0100E046F000E056F000E96
:10327000066F000E076F3DEC29F000C129F501C172
:103280002AF502C12BF503C12CF56BEC2EF00401DD
:103290004C0E826F5BEC0EF00401460E826F5BEC0D
:1032A0000EF004012C0E826F5BEC0EF025C500F1D0
:1032B00026C501F127C502F128C503F10101100E51
:1032C000046F000E056F000E066F000E076F5DECB9
:1032D00029F0CAEC29F02AC182F40401300E8227B9
:1032E0005BEC0EF02BC182F40401300E82275BEC04
:1032F0000EF02CC182F40401300E82275BEC0EF03C
:103300002DC182F40401300E82275BEC0EF02EC139
:1033100082F40401300E82275BEC0EF02FC182F4A0
:103320000401300E82275BEC0EF030C182F4040100
:10333000300E82275BEC0EF031C182F40401300EB6
:1033400082275BEC0EF032C182F40401300E82273A
:103350005BEC0EF033C182F40401300E82275BEC8B
:103360000EF014EF1AF00F9841EC2FF069EF23F0F4
:1033700004014C0E826F5BEC0EF00401350E826F7F
:103380005BEC0EF004012C0E826F5BEC0EF027EC70
:103390002AF00784B5C500F10794CAEC29F031C1C1
:1033A00082F40401300E82275BEC0EF032C182F40D
:1033B0000401300E82275BEC0EF033C182F404016D
:1033C000300E82275BEC0EF014EF1AF004EC2FF0B5
:1033D00027EC2AF033C500F1CAEC29F004014C0EA9
:1033E000826F5BEC0EF00401360E826F5BEC0EF028
:1033F00004012C0E826F5BEC0EF031C182F40401EB
:10340000300E82275BEC0EF032C182F40401300EE4
:1034100082275BEC0EF033C182F40401300E822768
:103420005BEC0EF014EF1AF065EC0EF069EF23F090
:1034300004014C0E826F5BEC0EF00401500E826FA3
:103440005BEC0EF004012C0E826F5BEC0EF085C37A
:103450002AF186C32BF187C32CF188C32DF189C3D0
:103460002EF18AC32FF18BC330F18CC331F18DC3A0
:1034700032F18EC333F1010175EC2AF0ECEC29F046
:1034800003018451530A0DE0030184514D0A38E0D1
:103490000401780E826F5BEC0EF065EC0EF069EFC4
:1034A00023F00401530E826F5BEC0EF0250E0C6EC0
:1034B00000C10BF002EC0BF0260E0C6E01C10BF0FC
:1034C00002EC0BF0270E0C6E02C10BF002EC0BF0BD
:1034D000280E0C6E03C10BF002EC0BF000C153F58B
:1034E00001C154F502C155F503C156F500C157F5A8
:1034F00001C158F502C159F503C15AF5F5EF1AF0AB
:1035000004014D0E826F5BEC0EF0290E0C6E00C1B3
:103510000BF002EC0BF000C15BF500C15CF5F5EFC0
:103520001AF004014C0E826F5BEC0EF00401540E95
:10353000826F5BEC0EF004012C0E826F5BEC0EF0E0
:1035400084C32AF185C32BF186C32CF187C32DF1E7
:1035500088C32EF189C32FF18AC330F18BC331F1B7
:103560008DC332F18EC333F1010175EC2AF0ECEC1E
:1035700029F00101000E046F000E056F010E066FA9
:10358000000E076F3DEC29F0210E0C6E00C10BF010
:1035900002EC0BF0220E0C6E01C10BF002EC0BF0F2
:1035A000230E0C6E02C10BF002EC0BF0240E0C6E1D
:1035B00003C10BF002EC0BF000C15DF501C15EF53B
:1035C00002C15FF503C160F5F5EF1AF004014C0E7E
:1035D000826F5BEC0EF00401490E826F5BEC0EF023
:1035E00004012C0E826F5BEC0EF0250E19EC0BF033
:1035F000E8CF00F1260E19EC0BF0E8CF01F1270E11
:1036000019EC0BF0E8CF02F1280E19EC0BF0E8CF23
:1036100003F1CAEC29F0ADEC27F00401730E826FC0
:103620005BEC0EF004012C0E826F5BEC0EF027ECCD
:103630002AF0290E19EC0BF0E8CF00F1CAEC29F0C2
:10364000ADEC27F00401730E826F5BEC0EF0040109
:103650002C0E826F5BEC0EF057C500F158C501F1DE
:1036600059C502F15AC503F1CAEC29F0ADEC27F0B7
:103670000401730E826F5BEC0EF004012C0E826F5E
:103680005BEC0EF027EC2AF05CC500F1CAEC29F0E7
:10369000ADEC27F004016D0E826F5BEC0EF00401BF
:1036A0002C0E826F5BEC0EF05DC500F15EC501F182
:1036B0005FC502F160C503F184EC23F004012C0E18
:1036C000826F5BEC0EF065EC0EF069EF23F083C3C4
:1036D0002AF184C32BF185C32CF186C32DF187C356
:1036E0002EF188C32FF189C330F18AC331F18BC326
:1036F00032F18CC333F1010175EC2AF0ECEC29F0C6
:10370000160E0C6E00C10BF002EC0BF0170E0C6ED7
:1037100001C10BF002EC0BF0180E0C6E02C10BF0A5
:1037200002EC0BF0190E0C6E03C10BF002EC0BF067
:1037300000C18AF101C18BF102C18CF103C18DF18D
:1037400000C18EF101C18FF102C190F103C191F16D
:1037500049EF1CF083C32AF184C32BF185C32CF1FC
:1037600086C32DF187C32EF188C32FF189C330F1B1
:103770008AC331F18BC332F18CC333F1010175EC93
:103780002AF0ECEC29F000C18AF101C18BF102C1F1
:103790008CF103C18DF100C18EF101C18FF102C125
:1037A00090F103C191F149EF1CF083C32AF184C366
:1037B0002BF185C32CF186C32DF187C32EF188C36D
:1037C0002FF189C330F18AC331F18CC332F18DC33B
:1037D00033F1010175EC2AF0ECEC29F00101000E47
:1037E000046F000E056F010E066F000E076F3DECB3
:1037F00029F01A0E0C6E00C10BF002EC0BF01B0E40
:103800000C6E01C10BF002EC0BF01C0E0C6E02C131
:103810000BF002EC0BF01D0E0C6E03C10BF002EC72
:103820000BF000C192F101C193F102C194F103C107
:1038300095F149EF1CF083C32AF184C32BF185C3B2
:103840002CF186C32DF187C32EF188C32FF189C3D4
:1038500030F18AC331F18CC332F18DC333F10101F0
:1038600075EC2AF0ECEC29F00101000E046F000E5B
:10387000056F010E066F000E076F3DEC29F000C1C9
:1038800092F101C193F102C194F103C195F149EFA5
:103890001CF0160E19EC0BF0E8CF00F1170E19EC26
:1038A0000BF0E8CF01F1180E19EC0BF0E8CF02F1A4
:1038B000190E19EC0BF0E8CF03F1CAEC29F0ADECCE
:1038C00027F00401730E826F5BEC0EF004012C0EE6
:1038D000826F5BEC0EF08AC100F18BC101F18CC1EB
:1038E00002F18DC103F1CAEC29F0ADEC27F004011F
:1038F000730E826F5BEC0EF004012C0E826F5BEC9A
:103900000EF01A0E19EC0BF0E8CF00F11B0E19ECBB
:103910000BF0E8CF01F11C0E19EC0BF0E8CF02F12F
:103920001D0E19EC0BF0E8CF03F184EC23F0040139
:103930002C0E826F5BEC0EF092C100F193C101F18D
:1039400094C102F195C103F184EC23F065EC0EF013
:1039500069EF23F00401690E826F5BEC0EF0040145
:103960002C0E826F5BEC0EF00101040E006F000E56
:10397000016F000E026F000E036FCAEC29F02CC11C
:1039800082F40401300E82275BEC0EF02DC182F42C
:103990000401300E82275BEC0EF02EC182F404018C
:1039A000300E82275BEC0EF02FC182F40401300E42
:1039B00082275BEC0EF030C182F40401300E8227C6
:1039C0005BEC0EF031C182F40401300E82275BEC17
:1039D0000EF032C182F40401300E82275BEC0EF04F
:1039E00033C182F40401300E82275BEC0EF0040137
:1039F0002C0E826F5BEC0EF00101060E006F000EC4
:103A0000016F000E026F000E036FCAEC29F02CC18B
:103A100082F40401300E82275BEC0EF02DC182F49B
:103A20000401300E82275BEC0EF02EC182F40401FB
:103A3000300E82275BEC0EF02FC182F40401300EB1
:103A400082275BEC0EF030C182F40401300E822735
:103A50005BEC0EF031C182F40401300E82275BEC86
:103A60000EF032C182F40401300E82275BEC0EF0BE
:103A700033C182F40401300E82275BEC0EF00401A6
:103A80002C0E826F5BEC0EF001012C0E006F000E0D
:103A9000016F000E026F000E036FCAEC29F02CC1FB
:103AA00082F40401300E82275BEC0EF02DC182F40B
:103AB0000401300E82275BEC0EF02EC182F404016B
:103AC000300E82275BEC0EF02FC182F40401300E21
:103AD00082275BEC0EF030C182F40401300E8227A5
:103AE0005BEC0EF031C182F40401300E82275BECF6
:103AF0000EF032C182F40401300E82275BEC0EF02E
:103B000033C182F40401300E82275BEC0EF0040115
:103B10002C0E826F5BEC0EF0200EF86EF76AF66AE0
:103B200004010900F5CF82F45BEC0EF00900F5CF3B
:103B300082F45BEC0EF00900F5CF82F45BEC0EF042
:103B40000900F5CF82F45BEC0EF00900F5CF82F4AA
:103B50005BEC0EF00900F5CF82F45BEC0EF009008F
:103B6000F5CF82F45BEC0EF00900F5CF82F45BEC4C
:103B70000EF065EC0EF069EF23F08351630AD8A4D0
:103B800069EF23F08451610AD8A469EF23F08551CD
:103B90006C0AD8A469EF23F08651410A3FE08651B0
:103BA000440A1BE08651420AD8B421EF1EF0865128
:103BB000350AD8B4F3EF24F08651360AD8B448EF6A
:103BC00025F08651370AD8B4B1EF25F08651380A6E
:103BD000D8B40FEF26F069EF23F00798079A040195
:103BE0007A0E826F5BEC0EF00401780E826F5BEC54
:103BF0000EF00401640E826F5BEC0EF00401550EB2
:103C0000826F5BEC0EF00AEF1EF004014C0E826F27
:103C10005BEC0EF065EC0EF069EF23F00788079A75
:103C200004017A0E826F5BEC0EF00401410E826F8C
:103C30005BEC0EF00401610E826F5BEC0EF0FEEFA8
:103C40001DF00798078A04017A0E826F5BEC0EF074
:103C50000401420E826F5BEC0EF00401610E826F74
:103C60005BEC0EF0FEEF1DF0010166673FEF1EF00A
:103C700067673FEF1EF068673FEF1EF0696715D07A
:103C80004F674AEF1EF050674AEF1EF051674AEF48
:103C90001EF052670AD00101000E006F000E016F86
:103CA000000E026F000E036F120011B80AD001015E
:103CB000620E046F010E056F000E066F000E076F97
:103CC00009D00101A70E046F020E056F000E066FEA
:103CD000000E076F66C100F167C101F168C102F112
:103CE00069C103F12CEC29F003BFE7EF1EF0119A34
:103CF000119C0101000E046FA80E056F550E066F92
:103D0000020E076F66C100F167C101F168C102F1DF
:103D100069C103F166C186F167C187F168C188F1A5
:103D200069C189F12CEC29F003BF0BD00101000E11
:103D3000866FA80E876F550E886F020E896F118AE5
:103D4000119C0E0E19EC0BF0E8CF18F10F0E19ECC8
:103D50000BF0E8CF19F1100E19EC0BF0E8CF1AF1C7
:103D6000110E19EC0BF0E8CF1BF175EC28F086C1B1
:103D700004F187C105F188C106F189C107F12CEC76
:103D800029F0078239EC28F075EC28F0079239EC1D
:103D900028F086C100F187C101F188C102F189C113
:103DA00003F1079239EC28F0CC0E046FE00E056F9A
:103DB000870E066F050E076F2CEC29F000C118F175
:103DC00001C119F102C11AF103C11BF13BD0119CD1
:103DD000119A0101800E006F1A0E016F060E026F1C
:103DE000000E036F4FC104F150C105F151C106F13E
:103DF00052C107F12CEC29F003AF05D027EC2AF0D3
:103E0000118C119A12000E0E19EC0BF0E8CF18F17C
:103E10000F0E19EC0BF0E8CF19F1100E19EC0BF0A6
:103E2000E8CF1AF1110E19EC0BF0E8CF1BF14FC1DE
:103E300000F150C101F151C102F152C103F10782F9
:103E400039EC28F018C100F119C101F11AC102F1D1
:103E50001BC103F112000401730E826F5BEC0EF0C4
:103E600004012C0E826F5BEC0EF0078462C166F1D8
:103E700063C167F164C168F165C169F14BC14FF17C
:103E80004CC150F14DC151F14EC152F157C159F1E0
:103E900058C15AF1079451EC1FF065EC0EF069EF30
:103EA00023F066C100F167C101F168C102F169C187
:103EB00003F10101CAEC29F0ADEC27F00401630E17
:103EC000826F5BEC0EF004012C0E826F5BEC0EF047
:103ED0004FC100F150C101F151C102F152C103F1D2
:103EE0000101CAEC29F0ADEC27F00401660E826FE7
:103EF0005BEC0EF004012C0E826F5BEC0EF027ECF5
:103F00002AF059C100F15AC101F10101CAEC29F0AE
:103F1000ADEC27F00401740E826F5BEC0EF0120022
:103F200010820401530E826F5BEC0EF004012C0E24
:103F3000826F5BEC0EF083C32AF184C32BF185C33F
:103F40002CF186C32DF187C32EF188C32FF189C3CD
:103F500030F18AC331F18BC332F18CC333F10101EB
:103F600075EC2AF0ECEC29F000C166F101C167F1B3
:103F700002C168F103C169F18EC32AF18FC32BF12D
:103F800090C32CF191C32DF192C32EF193C32FF165
:103F900094C330F195C331F196C332F197C333F135
:103FA000010175EC2AF0ECEC29F000C14FF101C1E0
:103FB00050F102C151F103C152F168EC2AF099C3EA
:103FC0002FF19AC330F19BC331F19CC332F19DC3F1
:103FD00033F1010175EC2AF0ECEC29F000C159F144
:103FE00001C15AF151EC1FF004012C0E826F5BEC01
:103FF0000EF008EF20F0118E18B0108C17BE02D012
:1040000017A4108E8251520A02E10F8201D00F9242
:104010008251750A02E1108401D010948251550A30
:1040200002E1108601D0109611A003D011A401D096
:104030001084078410B276EF20F010A462EF20F015
:10404000B6C166F1B7C167F1B8C168F1B9C169F12C
:10405000BAC16AF1BBC16BF1BCC16CF1BDC16DF1FC
:10406000BEC16EF1BFC16FF1C0C170F1C1C171F1CC
:10407000C2C172F1C3C173F1C4C174F1C5C175F19C
:10408000C6C176F1C7C177F1C8C178F1C9C179F16C
:10409000CAC17AF1CBC17BF1CCC17CF1CDC17DF13C
:1040A000CEC17EF1CFC17FF1D0C180F1D1C181F10C
:1040B000D2C182F1D3C183F1D4C184F1D5C185F1DC
:1040C0006AEF20F062C166F163C167F164C168F113
:1040D00065C169F14BC14FF14CC150F14DC151F176
:1040E0004EC152F157C159F158C15AF107940FA06E
:1040F00098EF20F00101926785EF20F0936785EF3C
:1041000020F0946785EF20F0956789EF20F098EF15
:1041100020F034EC1EF092C104F193C105F194C17A
:1041200006F195C107F12CEC29F003BF2FEF23F026
:1041300034EC1EF00101000E046F000E056F010E3D
:10414000066F000E076F5DEC29F011A02CD011A2B4
:104150002AD0CAEC29F0296701D007D004012D0E1E
:10416000826F5BEC0EF02DEF23F030C182F404017E
:10417000300E82275BEC0EF031C182F40401300E68
:1041800082275BEC0EF032C182F40401300E8227EC
:104190005BEC0EF033C182F40401300E82275BEC3D
:1041A0000EF02DEF23F012A8C5D0129819C01AF006
:1041B0001A3A1A42070E1A1600011A50000AD8B409
:1041C00066EF21F000011A50010AD8B4F2EF20F096
:1041D00000011A50020AD8B4F0EF20F098EF21F055
:1041E00098EF21F027EC2AF029C001F12AC000F154
:1041F000D89001330033D890013300330101630EAE
:10420000046F000E056F000E066F000E076F5DEC69
:1042100029F0280E046F000E056F000E066F000EC9
:10422000076F2CEC29F000C12CF027EC2AF027C0F6
:1042300001F1019F019D28C000F10101A40E046F4E
:10424000000E056F000E066F000E076F5DEC29F083
:1042500000C12BF000C104F101C105F102C106F15A
:1042600003C107F1640E006F000E016F000E026FB4
:10427000000E036F2CEC29F0050E046F000E056F85
:10428000000E066F000E076F5DEC29F000C104F10F
:1042900001C105F102C106F103C107F127EC2AF0C3
:1042A0002CC000F12CEC29F000C12DF02DC0E8FF4E
:1042B000050F2C5C03E78A8498EF21F02DC0E8FFFE
:1042C0000A0F2C5C01E68A9498EF21F000C124F1DA
:1042D00001C125F102C126F103C127F127EC2AF023
:1042E0002DEC2AF019501F0BE8CF00F10101640EEC
:1042F000046F000E056F000E066F000E076F3DEC99
:1043000029F024C104F125C105F126C106F127C118
:1043100007F12CEC29F003BF02D08A9401D08A84E3
:1043200024C100F125C101F126C102F127C103F129
:104330002FEF23F000C124F101C125F102C126F1C4
:1043400003C127F110AE4CD0109E00C108F101C18D
:1043500009F102C10AF103C10BF1CAEC29F030C125
:10436000D6F131C1D7F132C1D8F133C1D9F108C189
:1043700000F109C101F10AC102F10BC103F1010110
:104380006C0E046F070E056F000E066F000E076FB0
:104390002CEC29F003BF04D00101550EDA6F1CD0BC
:1043A00008C100F109C101F10AC102F10BC103F119
:1043B0000101A40E046F060E056F000E066F000EBD
:1043C000076F2CEC29F003BF04D001017F0EDA6FD8
:1043D00003D00101FF0EDA6F1B8E11AE2FEF23F019
:1043E00024C100F125C101F126C102F127C103F169
:1043F00010A402EF22F00401750E826F5BEC0EF048
:1044000007EF22F00401720E826F5BEC0EF00401E4
:104410002C0E826F5BEC0EF0CAEC29F0296716EFC8
:1044200022F00401200E826F19EF22F004012D0EFC
:10443000826F5BEC0EF030C182F40401300E8227F3
:104440005BEC0EF031C182F40401300E82275BEC8C
:104450000EF004012E0E826F5BEC0EF032C182F47E
:104460000401300E82275BEC0EF033C182F40401AC
:10447000300E82275BEC0EF004016D0E826F5BEC58
:104480000EF004012C0E826F5BEC0EF04FC100F1B8
:1044900050C101F151C102F152C103F10101CAEC55
:1044A00029F0ADEC27F00401480E826F5BEC0EF0B2
:1044B00004017A0E826F5BEC0EF004012C0E826F09
:1044C0005BEC0EF066C100F167C101F168C102F159
:1044D00069C103F10101CAEC29F0ADEC27F0040138
:1044E000630E826F5BEC0EF004012C0E826F5BECAE
:1044F0000EF066C100F167C101F168C102F169C146
:1045000003F101010A0E046F000E056F000E066F25
:10451000000E076F3DEC29F0000E046F120E056FC0
:10452000000E066F000E076F5DEC29F0CAEC29F053
:104530002AC182F40401300E82275BEC0EF02BC1FD
:1045400082F40401300E82275BEC0EF02CC182F461
:104550000401300E82275BEC0EF02DC182F40401C1
:10456000300E82275BEC0EF02EC182F40401300E77
:1045700082275BEC0EF02FC182F40401300E8227FB
:104580005BEC0EF030C182F40401300E82275BEC4C
:104590000EF004012E0E826F5BEC0EF031C182F43E
:1045A0000401300E82275BEC0EF032C182F404016C
:1045B000300E82275BEC0EF033C182F40401300E22
:1045C00082275BEC0EF00401730E826F5BEC0EF041
:1045D00004012C0E826F5BEC0EF027EC2AF059C11F
:1045E00000F15AC101F193EC24F00FB2FBEF22F07D
:1045F0000FA02DEF23F004012C0E826F5BEC0EF068
:10460000200EF86EF76AF66A04010900F5CF82F40D
:104610005BEC0EF00900F5CF82F45BEC0EF00900C4
:10462000F5CF82F45BEC0EF00900F5CF82F45BEC81
:104630000EF00900F5CF82F45BEC0EF00900F5CF27
:1046400082F45BEC0EF00900F5CF82F45BEC0EF027
:104650000900F5CF82F45BEC0EF065EC0EF00F90E4
:1046600069EF23F00401630E826F5BEC0EF004012E
:104670002C0E826F5BEC0EF06FEC23F004012C0E1D
:10468000826F5BEC0EF0E2EC23F004012C0E826FE3
:104690005BEC0EF05EEC24F004012C0E826F5BEC00
:1046A0000EF00101F80E006FCD0E016F660E026F65
:1046B000030E036F84EC23F004012C0E826F5BEC7D
:1046C0000EF074EC24F065EC0EF069EF23F065EC6D
:1046D0000EF00301C26B0790109278EF26F0D8908D
:1046E0000E0E19EC0BF0E8CF00F10F0E19EC0BF0E9
:1046F000E8CF01F1100E19EC0BF0E8CF02F1110E2A
:1047000019EC0BF0E8CF03F10101000E046F000E6D
:10471000056F010E066F000E076F5DEC29F0CAEC05
:1047200029F02AC182F40401300E82275BEC0EF0DE
:104730002BC182F40401300E82275BEC0EF02CC1F9
:1047400082F40401300E82275BEC0EF02DC182F45E
:104750000401300E82275BEC0EF02EC182F40401BE
:10476000300E82275BEC0EF02FC182F40401300E74
:1047700082275BEC0EF030C182F40401300E8227F8
:104780005BEC0EF031C182F40401300E82275BEC49
:104790000EF004012E0E826F5BEC0EF032C182F43B
:1047A0000401300E82275BEC0EF033C182F4040169
:1047B000300E82275BEC0EF004016D0E826F5BEC15
:1047C0000EF01200120E19EC0BF0E8CF00F1130EF0
:1047D00019EC0BF0E8CF01F1140E19EC0BF0E8CF57
:1047E00002F1150E19EC0BF0E8CF03F101010A0EEE
:1047F000046F000E056F000E066F000E076F3DEC94
:1048000029F0000E046F120E056F000E066F000EE9
:10481000076F5DEC29F0CAEC29F02AC182F404018B
:10482000300E82275BEC0EF02BC182F40401300EB7
:1048300082275BEC0EF02CC182F40401300E82273B
:104840005BEC0EF02DC182F40401300E82275BEC8C
:104850000EF02EC182F40401300E82275BEC0EF0C4
:104860002FC182F40401300E82275BEC0EF030C1C0
:1048700082F40401300E82275BEC0EF004012E0E50
:10488000826F5BEC0EF031C182F40401300E82279E
:104890005BEC0EF032C182F40401300E82275BEC37
:1048A0000EF033C182F40401300E82275BEC0EF06F
:1048B0000401730E826F5BEC0EF012000A0E19EC0D
:1048C0000BF0E8CF00F10B0E19EC0BF0E8CF01F183
:1048D0000C0E19EC0BF0E8CF02F10D0E19EC0BF0F9
:1048E000E8CF03F193EF24F0060E19EC0BF0E8CFBC
:1048F00000F1070E19EC0BF0E8CF01F1080E19ECEE
:104900000BF0E8CF02F1090E19EC0BF0E8CF03F140
:1049100093EF24F0010127EC2AF0078457C100F13E
:1049200058C101F107940101E80E046F800E056F74
:10493000000E066F000E076F3DEC29F0000E046FAD
:10494000040E056F000E066F000E076F5DEC29F078
:10495000880E046F130E056F000E066F000E076FB2
:104960002CEC29F00A0E046F000E056F000E066F86
:10497000000E076F5DEC29F0CAEC29F001012967F0
:10498000C7EF24F00401200E826FCAEF24F0040167
:104990002D0E826F5BEC0EF030C182F40401300EFC
:1049A00082275BEC0EF031C182F40401300E8227C5
:1049B0005BEC0EF032C182F40401300E82275BEC16
:1049C0000EF004012E0E826F5BEC0EF033C182F408
:1049D0000401300E82275BEC0EF00401430E826F5F
:1049E0005BEC0EF0120087C32AF188C32BF189C358
:1049F0002CF18AC32DF18BC32EF18CC32FF18DC303
:104A000030F18EC331F190C332F191C333F1010122
:104A1000296B75EC2AF0ECEC29F00101000E046F13
:104A2000000E056F010E066F000E076F3DEC29F0BA
:104A30000E0E0C6E00C10BF002EC0BF00F0E0C6EA4
:104A400001C10BF002EC0BF0100E0C6E02C10BF06A
:104A500002EC0BF0110E0C6E03C10BF002EC0BF02C
:104A600004017A0E826F5BEC0EF004012C0E826F53
:104A70005BEC0EF00401350E826F5BEC0EF004016E
:104A80002C0E826F5BEC0EF06FEC23F00AEF1EF041
:104A900087C32AF188C32BF189C32CF18AC32DF176
:104AA0008BC32EF18CC32FF18DC330F18EC331F146
:104AB00090C332F191C333F10101296B75EC2AF0F7
:104AC000ECEC29F0880E046F130E056F000E066FD4
:104AD000000E076F31EC29F0000E046F040E056F15
:104AE000000E066F000E076F3DEC29F00101E80E85
:104AF000046F800E056F000E066F000E076F5DECF1
:104B000029F00A0E0C6E00C10BF002EC0BF00B0E3C
:104B10000C6E01C10BF002EC0BF00C0E0C6E02C11E
:104B20000BF002EC0BF00D0E0C6E03C10BF002EC5F
:104B30000BF004017A0E826F5BEC0EF004012C0E78
:104B4000826F5BEC0EF00401360E826F5BEC0EF0B0
:104B500004012C0E826F5BEC0EF05EEC24F00AEF89
:104B60001EF087C32AF188C32BF189C32CF18AC3B5
:104B70002DF18BC32EF18CC32FF18DC330F18FC378
:104B800031F190C332F191C333F1010175EC2AF098
:104B9000ECEC29F0000E046F120E056F000E066F8C
:104BA000000E076F3DEC29F001010A0E046F000EA4
:104BB000056F000E066F000E076F5DEC29F0120EF8
:104BC0000C6E00C10BF002EC0BF0130E0C6E01C169
:104BD0000BF002EC0BF0140E0C6E02C10BF002ECA9
:104BE0000BF0150E0C6E03C10BF002EC0BF0040180
:104BF0007A0E826F5BEC0EF004012C0E826F5BEC80
:104C00000EF00401370E826F5BEC0EF004012C0EE7
:104C1000826F5BEC0EF0E2EC23F00AEF1EF087C32C
:104C20002AF188C32BF189C32CF18AC32DF18BC3E0
:104C30002EF18CC32FF18DC330F18EC331F190C3AF
:104C400032F191C333F10101296B75EC2AF0ECECE0
:104C500029F0880E046F130E056F000E066F000E0C
:104C6000076F31EC29F0000E046F040E056F000E83
:104C7000066F000E076F3DEC29F00101E80E046F8E
:104C8000800E056F000E066F000E076F5DEC29F0B9
:104C9000060E0C6E00C10BF002EC0BF0070E0C6E52
:104CA00001C10BF002EC0BF0080E0C6E02C10BF010
:104CB00002EC0BF0090E0C6E03C10BF002EC0BF0D2
:104CC00004017A0E826F5BEC0EF004012C0E826FF1
:104CD0005BEC0EF00401380E826F5BEC0EF0040109
:104CE0002C0E826F5BEC0EF074EC24F00AEF1EF0D9
:104CF00007A8ECEF26F00101800E006F1A0E016F7D
:104D0000060E026F000E036F4BC104F14CC105F19A
:104D10004DC106F14EC107F12CEC29F003BF33EF72
:104D200027F0A7EC27F04BC100F14CC101F14DC1B8
:104D300002F14EC103F1078239EC28F018C104F1E9
:104D400019C105F11AC106F11BC107F1F80E006F78
:104D5000CD0E016F660E026F030E036F2CEC29F06F
:104D60000E0E0C6E00C10BF002EC0BF00F0E0C6E71
:104D700001C10BF002EC0BF0100E0C6E02C10BF037
:104D800002EC0BF0110E0C6E03C10BF002EC0BF0F9
:104D90000784010127EC2AF057C100F158C101F145
:104DA00007940A0E0C6E00C10BF002EC0BF00B0E18
:104DB0000C6E01C10BF002EC0BF00C0E0C6E02C17C
:104DC0000BF002EC0BF00D0E0C6E03C10BF002ECBD
:104DD0000BF0079833EF27F007AA33EF27F007848B
:104DE000010127EC2AF057C100F158C101F10794E5
:104DF000060E0C6E00C10BF002EC0BF0070E0C6EF1
:104E000001C10BF002EC0BF0080E0C6E02C10BF0AE
:104E100002EC0BF0090E0C6E03C10BF002EC0BF070
:104E2000078462C100F163C101F164C102F165C18F
:104E300003F10794120E0C6E00C10BF002EC0BF0A4
:104E4000130E0C6E01C10BF002EC0BF0140E0C6E85
:104E500002C10BF002EC0BF0150E0C6E03C10BF04F
:104E600002EC0BF0079A0401805181197F0B0BE0D3
:104E70009EA809D014EE00F081517F0BE126E75087
:104E8000812B0F01AD6E05012F51010A13E081AA9C
:104E90005AEF27F005012F51000A0AE00FB85AEF28
:104EA00027F0050130675AEF27F00FB85AEF27F0C7
:104EB000C9EF30F081B86FEF27F057EC2BF0050108
:104EC0002F51020A02E06FEF27F05C2F6FEF27F0FF
:104ED0005BC55CF50501010E306F3C0E316FAFEF25
:104EE0000DF018C100F119C101F11AC102F11BC185
:104EF00003F1000E046F000E056F010E066F000E29
:104F0000076F5DEC29F029A19CEF27F02051D8B460
:104F10009CEF27F018C100F119C101F11AC102F18B
:104F20001BC103F1000E046F000E056F0A0E066F21
:104F3000000E076F5DEC29F012000101045100130F
:104F40000551011306510213075103131200010109
:104F5000186B196B1A6B1B6B12002AC182F40401C7
:104F6000300E82275BEC0EF02BC182F40401300E70
:104F700082275BEC0EF02CC182F40401300E8227F4
:104F80005BEC0EF02DC182F40401300E82275BEC45
:104F90000EF02EC182F40401300E82275BEC0EF07D
:104FA0002FC182F40401300E82275BEC0EF030C179
:104FB00082F40401300E82275BEC0EF031C182F4E2
:104FC0000401300E82275BEC0EF032C182F4040142
:104FD000300E82275BEC0EF033C182F40401300EF8
:104FE00082275BEC0EF012002FC182F40401300E18
:104FF00082275BEC0EF030C182F40401300E822770
:105000005BEC0EF031C182F40401300E82275BECC0
:105010000EF032C182F40401300E82275BEC0EF0F8
:1050200033C182F40401300E82275BEC0EF01200D3
:10503000060E1D6E060E1E6E060E1F6E1D2E1EEF38
:1050400028F01E2E1EEF28F01F2E1EEF28F08B8456
:10505000020E1D6E020E1E6E020E1F6E1D2E2EEF14
:1050600028F01E2E2EEF28F01F2E2EEF28F08B9406
:1050700012000101005305E1015303E1025301E174
:10508000002BFCEC28F027EC2AF03951006F3A5144
:10509000016F420E046F4B0E056F000E066F000E7F
:1050A000076F3DEC29F000C104F101C105F102C117
:1050B00006F103C107F118C100F119C101F11AC1CC
:1050C00002F11BC103F107B26AEF28F031EC29F0BD
:1050D0006CEF28F02CEC29F000C118F101C119F196
:1050E00002C11AF103C11BF1120027EC2AF059C1C9
:1050F00000F15AC101F1060E19EC0BF0E8CF04F1F2
:10510000070E19EC0BF0E8CF05F1080E19EC0BF0C7
:10511000E8CF06F1090E19EC0BF0E8CF07F12CEC03
:1051200029F000C124F101C125F102C126F103C11A
:1051300027F1290E046F000E056F000E066F000E9A
:10514000076F3DEC29F0EE0E046F430E056F000E65
:10515000066F000E076F31EC29F024C104F125C160
:1051600005F126C106F127C107F13DEC29F000C188
:105170001CF101C11DF102C11EF103C11FF1120E8C
:1051800019EC0BF0E8CF04F1130E19EC0BF0E8CF9B
:1051900005F1140E19EC0BF0E8CF06F1150E19EC21
:1051A0000BF0E8CF07F10D0E006F000E016F000E3F
:1051B000026F000E036F3DEC29F0180E046F000E15
:1051C000056F000E066F000E076F5DEC29F01CC125
:1051D00004F11DC105F11EC106F11FC107F131EC3B
:1051E00029F06A0E046F2A0E056F000E066F000E7E
:1051F000076F2CEC29F01200BF0EFA6E200E3A6FEA
:10520000396BD8900037013702370337D8B00DEF2C
:1052100029F03A2F02EF29F039073A070353D8B49F
:1052200012000331070B80093F6F03390F0B010F89
:10523000396F80EC5FF0406F390580EC5FF0405DC6
:10524000405F396B3F33D8B0392739333FA922EF5C
:1052500029F040513927120001014CEC2AF0D8B056
:105260001200010103510719346F0FEC2AF0D89096
:105270000751031934AF800F12000101346B33EC76
:105280002AF0D8A049EC2AF0D8B012001EEC2AF07F
:1052900027EC2AF01F0E366F5FEC2AF00B35D8B0E2
:1052A0000FEC2AF0D8A00335D8B01200362F4CEFFF
:1052B00029F034B136EC2AF012000101346B0451AC
:1052C0000511061107110008D8A033EC2AF0D8A068
:1052D00049EC2AF0D8B01200086B096B0A6B0B6B13
:1052E0005FEC2AF01F0E366F5FEC2AF007510B5D62
:1052F000D8A487EF29F006510A5DD8A487EF29F0DA
:105300000551095DD8A487EF29F00451085DD8A0A4
:105310009AEF29F00451085F0551D8A0053D095FB7
:105320000651D8A0063D0A5F0751D8A0073D0B5F84
:10533000D8900081362F74EF29F034B136EC2AF082
:10534000346B33EC2AF0D89063EC2AF007510B5DF4
:10535000D8A4B7EF29F006510A5DD8A4B7EF29F019
:105360000551095DD8A4B7EF29F00451085DD8A014
:10537000C6EF29F0003FC6EF29F0013FC6EF29F044
:10538000023FC6EF29F0032BD8B4120034B136EC3B
:105390002AF012000101346B33EC2AF0D8B012006D
:1053A00068EC2AF0200E366F0037013702370337DA
:1053B00011EE33F00A0E376FE7360A0EE75CD8B00D
:1053C000E76EE552372FDCEF29F0362FD4EF29F0C6
:1053D00034B12981D890120001010A0E346F200ED9
:1053E000366F11EE29F03451376F0A0ED890E6521D
:1053F000D8B0E726E732372FF7EF29F0033302332F
:1054000001330033362FF1EF29F0E750FF0FD8A01A
:105410000335D8B0120029B136EC2AF0120004513D
:1054200000270551D8B0053D01270651D8B0063DEB
:1054300002270751D8B0073D032712000051086F1B
:105440000151096F02510A6F03510B6F12000101E4
:10545000006B016B026B036B12000101046B056BA7
:10546000066B076B12000335D8A012000351800BA6
:10547000001F011F021F031F003F46EF2AF0013FDC
:1054800046EF2AF0023F46EF2AF0032B342B032588
:1054900012000735D8A012000751800B041F051F0A
:1054A000061F071F043F5CEF2AF0053F5CEF2AF060
:1054B000063F5CEF2AF0072B342B0725120000373C
:1054C000013702370337083709370A370B3712001D
:1054D0000101296B2A6B2B6B2C6B2D6B2E6B2F6BA9
:1054E000306B316B326B336B120001012A510F0BA1
:1054F0002A6F2B510F0B2B6F2C510F0B2C6F2D5133
:105500000F0B2D6F2E510F0B2E6F2F510F0B2F6F77
:1055100030510F0B306F31510F0B316F32510F0B78
:10552000326F33510F0B336F120010A806D08994DD
:10553000000EC76E220EC66E05D08984000EC76E9F
:10554000220EC66E050EE82EFED7120010A802D05D
:10555000898401D08994050EE82EFED7120095ECBF
:105560002AF09E96C69E000EC96EFF0E9EB602D011
:10557000E82EFCD79E96C69E000EC96EFF0E9EB604
:1055800002D0E82EFCD7C9CFABF59E96C69E000E82
:10559000C96EFF0E9EB602D0E82EFCD7C9CFACF57F
:1055A0009E96C69E000EC96EFF0E9EB602D0E82ED5
:1055B000FCD7C9CFADF59E96C69E000EC96EFF0EF4
:1055C0009EB602D0E82EFCD7C9CFAEF59E96C69EF9
:1055D000000EC96EFF0E9EB602D0E82EFCD7C9CFD2
:1055E000AFF59E96C69E000EC96EFF0E9EB602D007
:1055F000E82EFCD7C9CFB0F59E96C69E000EC96EA8
:10560000FF0E9EB602D0E82EFCD7C9CFB1F5A6ECAE
:105610002AF0120095EC2AF09E96C69E800EC96E66
:10562000FF0E9EB602D0E82EFCD79E96C69EABC556
:10563000C9FFFF0E9EB602D0E82EFCD79E96C69EEE
:10564000ACC5C9FFFF0E9EB602D0E82EFCD79E96D1
:10565000C69EADC5C9FFFF0E9EB602D0E82EFCD790
:105660009E96C69EAEC5C9FFFF0E9EB602D0E82E1E
:10567000FCD79E96C69EAFC5C9FFFF0E9EB602D050
:10568000E82EFCD79E96C69EB0C5C9FFFF0E9EB6FB
:1056900002D0E82EFCD79E96C69EB1C5C9FFFF0E6C
:1056A0009EB602D0E82EFCD7A6EC2AF0120095ECAC
:1056B0002AF09E96C69E070EC96EFF0E9EB602D0B9
:1056C000E82EFCD79E96C69E000EC96EFF0E9EB6B3
:1056D00002D0E82EFCD7C9CFABF59E96C69E000E31
:1056E000C96EFF0E9EB602D0E82EFCD7C9CFACF52E
:1056F0009E96C69E000EC96EFF0E9EB602D0E82E84
:10570000FCD7C9CFADF59E96C69E000EC96EFF0EA2
:105710009EB602D0E82EFCD7C9CFAEF5A6EC2AF093
:1057200095EC2AF09E96C69E21C0C9FFFF0E9EB63C
:1057300002D0E82EFCD79E96C69E000EC96EFF0EC4
:105740009EB602D0E82EFCD7C9CFB2F5A6EC2AF05F
:10575000120095EC2AF09E96C69E870EC96EFF0E2B
:105760009EB602D0E82EFCD79E96C69EABC5C9FF5A
:10577000FF0E9EB602D0E82EFCD79E96C69EACC504
:10578000C9FFFF0E9EB602D0E82EFCD79E96C69E9D
:10579000ADC5C9FFFF0E9EB602D0E82EFCD79E967F
:1057A000C69EAEC5C9FFFF0E9EB602D0E82EFCD73E
:1057B000A6EC2AF095EC2AF09E96C69E22C0C9FF60
:1057C000FF0E9EB602D0E82EFCD79E96C69EB2C5AE
:1057D000C9FFFF0E9EB602D0E82EFCD7A6EC2AF039
:1057E000120095EC2AF09E96C69E870EC96EFF0E9B
:1057F0009EB602D0E82EFCD79E96C69E000EC96EBD
:10580000FF0E9EB602D0E82EFCD79E96C69E800E56
:10581000C96EFF0E9EB602D0E82EFCD79E96C69E9D
:10582000800EC96EFF0E9EB602D0E82EFCD79E9663
:10583000C69E800EC96EFF0E9EB602D0E82EFCD723
:10584000A6EC2AF0120095EC2AF09E96C69E870ED2
:10585000C96EFF0E9EB602D0E82EFCD79E96C69E5D
:10586000000EC96EFF0E9EB602D0E82EFCD79E96A3
:10587000C69E000EC96EFF0E9EB602D0E82EFCD763
:105880009E96C69E800EC96EFF0E9EB602D0E82E72
:10589000FCD79E96C69E800EC96EFF0E9EB602D0A5
:1058A000E82EFCD7A6EC2AF0120010A82DD095EC1B
:1058B0002AF09E96C69E22C0C9FFFF0E9EB602D059
:1058C000E82EFCD79E96C69E450EC96EFF0E9EB66C
:1058D00002D0E82EFCD7A6EC2AF095EC2AF09E9692
:1058E000C69E8F0EC96EFF0E9EB602D0E82EFCD764
:1058F0009E96C69E000EC96EFF0E9EB602D0E82E82
:10590000FCD7A6EC2AF0120095EC2AF09E96C69ED3
:1059100022C0C9FFFF0E9EB602D0E82EFCD79E968D
:10592000C69E010EC96EFF0E9EB602D0E82EFCD7B1
:10593000A6EC2AF095EC2AF09E96C69E910EC96EB2
:10594000FF0E9EB602D0E82EFCD79E96C69EA50EF0
:10595000C96EFF0E9EB602D0E82EFCD7A6EC2AF048
:10596000120095EC2AF09E96C69E22C0C9FFFF0E3B
:105970009EB602D0E82EFCD79E96C69E810EC96EBA
:10598000FF0E9EB602D0E82EFCD7A6EC2AF012003D
:1059900095EC2AF09E96C69E22C0C9FFFF0E9EB6C9
:1059A00002D0E82EFCD79E96C69E010EC96EFF0E51
:1059B0009EB602D0E82EFCD7A6EC2AF0120095EC99
:1059C0002AF09E96C69E910EC96EFF0E9EB602D01C
:1059D000E82EFCD79E96C69EA50EC96EFF0E9EB6FB
:1059E00002D0E82EFCD7A6EC2AF0120095EC2AF0A3
:1059F0009E96C69E910EC96EFF0E9EB602D0E82EF0
:105A0000FCD79E96C69E000EC96EFF0E9EB602D0B3
:105A1000E82EFCD7A6EC2AF012000501256B266BB8
:105A2000276B286B899A400EC76E200EC66E9E9615
:105A3000C69E030EC96EFF0E9EB602D0E82EFCD79E
:105A40009E96C69E27C5C9FFFF0E9EB602D0E82EC1
:105A5000FCD79E96C69E26C5C9FFFF0E9EB602D0F5
:105A6000E82EFCD79E96C69E25C5C9FFFF0E9EB6A2
:105A700002D0E82EFCD79E96C69EC952FF0E9EB657
:105A800002D0E82EFCD7898A0F01C950FF0A01E134
:105A9000120005012E51130A05E005012E51170AC7
:105AA0000CE012000501F00E256FFF0E266F0F0EA1
:105AB000276F000E286F66EF2DF00501F00E256FA1
:105AC000FF0E266FFF0E276F000E286F899A400E7B
:105AD000C76E200EC66E9E96C69E030EC96EFF0E42
:105AE0009EB602D0E82EFCD79E96C69E27C5C9FF5B
:105AF000FF0E9EB602D0E82EFCD79E96C69E26C507
:105B0000C9FFFF0E9EB602D0E82EFCD79E96C69E19
:105B100025C5C9FFFF0E9EB602D0E82EFCD79E9683
:105B2000C69EC952FF0E9EB602D0E82EFCD7898AC7
:105B30000F01C950FF0A1DE005012E51130A05E0AF
:105B400005012E51170A0BE012000501000E256F0A
:105B5000000E266F100E276F000E286F1200050131
:105B6000000E256F000E266F000E276F010E286FA6
:105B700012000501256B266B276B286B05012E5142
:105B8000130A05E005012E51170A0CE01200050169
:105B9000000E216F000E226F080E236F000E246F7F
:105BA000DBEF2DF00501000E216F000E226F800E3D
:105BB000236F000E246F21C500F122C501F123C51A
:105BC00002F124C503F125C504F126C505F127C559
:105BD00006F128C507F19DEC27F000C125F501C1AC
:105BE00026F502C127F503C128F5899A400EC76E34
:105BF000200EC66E9E96C69E030EC96EFF0E9EB602
:105C000002D0E82EFCD79E96C69E27C5C9FFFF0E80
:105C10009EB602D0E82EFCD79E96C69E26C5C9FF2A
:105C2000FF0E9EB602D0E82EFCD79E96C69E25C5D6
:105C3000C9FFFF0E9EB602D0E82EFCD79E96C69EE8
:105C4000C952FF0E9EB602D0E82EFCD7898AC950F1
:105C5000FF0A08E104C125F505C126F506C127F5AF
:105C600007C128F5D890050124332333223321338B
:105C70002151F00B216F216745EF2EF0226745EF90
:105C80002EF0236745EF2EF02467DBEF2DF00501A2
:105C9000100E2527E86A2623E86A2723E86A2823C6
:105CA0001200E86A05012E51130A06E005012E5183
:105CB000170A0BE0020E120005012851000A03E149
:105CC0002751F00B07E0010E120005012851000AD0
:105CD00001E0010E120029C500F12AC501F12BC512
:105CE00002F12CC503F125C504F126C505F127C530
:105CF00006F128C507F12CEC29F003BF120051EC86
:105D00002EF0D8A4E3EF2EF0899A400EC76E200E35
:105D1000C66E9E96C69E060EC96EFF0E9EB602D039
:105D2000E82EFCD7898A899A9E96C69E020EC96E75
:105D3000FF0E9EB602D0E82EFCD79E96C69E27C5C3
:105D4000C9FFFF0E9EB602D0E82EFCD79E96C69ED7
:105D500026C5C9FFFF0E9EB602D0E82EFCD79E9640
:105D6000C69E25C5C9FFFF0E9EB602D0E82EFCD701
:105D70009E96C69E000EC96EFF0E9EB602D0E82EFD
:105D8000FCD7898A899A9E96C69E050EC96EFF0E1B
:105D90009EB602D0E82EFCD79E96C69EC952FF0E34
:105DA0009EB602D0E82EFCD7C9B0CCEF2EF0898A7F
:105DB0000501100E2527E86A2623E86A2723E86AEA
:105DC00028236BEF2EF01200899A400EC76E200E2A
:105DD000C66E9E96C69E060EC96EFF0E9EB602D079
:105DE000E82EFCD7898A899A9E96C69EC70EC96EF0
:105DF000FF0E9EB602D0E82EFCD7898A0501256BDE
:105E0000266B276B286B1200899A400EC76E200EF6
:105E1000C66E9E96C69E050EC96EFF0E9EB602D039
:105E2000E82EFCD79E96C69EC952FF0E9EB602D0A3
:105E3000E82EFCD7C9CF33F5898A1200899A400E23
:105E4000C76E200EC66E9E96C69EB90EC96EFF0E18
:105E50009EB602D0E82EFCD7898A1200899A400E9D
:105E6000C76E200EC66E9E96C69EAB0EC96EFF0E06
:105E70009EB602D0E82EFCD7898AFF0EE82EFED708
:105E8000120051EC2EF0D8A41200899A400EC76E71
:105E9000200EC66E9E96C69E030EC96EFF0E9EB65F
:105EA00002D0E82EFCD79E96C69E27C5C9FFFF0EDE
:105EB0009EB602D0E82EFCD79E96C69E26C5C9FF88
:105EC000FF0E9EB602D0E82EFCD79E96C69E25C534
:105ED000C9FFFF0E9EB602D0E82EFCD79E96C69E46
:105EE000C952FF0E9EB602D0E82EFCD7898A0F0158
:105EF000C950FF0AD8A43CEF30F00501FE0E336F05
:105F0000AFEC2AF0ABC534F5ACC535F5ADC536F50B
:105F1000AEC537F5AFC538F5B0C539F5B1C53AF5F9
:105F20000784B6C166F1B7C167F1B8C168F1B9C1FC
:105F300069F14BC14FF14CC150F14DC151F14EC10E
:105F400052F157C159F158C15AF134EC1EF000C159
:105F50003BF501C13CF502C13DF503C13EF505012C
:105F60005D67BAEF2FF05E67BAEF2FF05F67BAEFA9
:105F70002FF06067BEEF2FF0CBEF2FF05DC504F17F
:105F80005EC505F15FC506F160C507F12CEC29F08F
:105F900003BF3CEF30F059C13FF55AC140F5B5C5DC
:105FA00041F5B6C542F507940501110E326F899A85
:105FB000400EC76E200EC66E9E96C69E060EC96E19
:105FC000FF0E9EB602D0E82EFCD7898A899A9E964B
:105FD000C69E020EC96EFF0E9EB602D0E82EFCD7FA
:105FE0009E96C69E27C5C9FFFF0E9EB602D0E82E1C
:105FF000FCD79E96C69E26C5C9FFFF0E9EB602D050
:10600000E82EFCD79E96C69E25C5C9FFFF0E9EB6FC
:1060100002D0E82EFCD725EE33F0322F02D01CEF51
:1060200030F09E96C69EDECFC9FFFF0E9EB602D010
:10603000E82EFCD70DEF30F0898A899A9E96C69E8D
:10604000050EC96EFF0E9EB602D0E82EFCD79E96B6
:10605000C69EC952FF0E9EB602D0E82EFCD7C9B02C
:1060600027EF30F0898A0501100E2527E86A2623DC
:10607000E86A2723E86A2823120021C500F122C517
:1060800001F123C502F124C503F1899A400EC76EC0
:10609000200EC66E9E96C69E0B0EC96EFF0E9EB655
:1060A00002D0E82EFCD79E96C69E02C1C9FFFF0E05
:1060B0009EB602D0E82EFCD79E96C69E01C1C9FFAF
:1060C000FF0E9EB602D0E82EFCD79E96C69E00C15B
:1060D000C9FFFF0E9EB602D0E82EFCD79E96C69E44
:1060E000C952FF0E9EB602D0E82EFCD725EE33F043
:1060F0000501100E326F9E96C69EC952FF0E9EB6C7
:1061000002D0E82EFCD7C9CFDEFF322F7BEF30F074
:10611000898A1200899A400EC76E200EC66E9E961E
:10612000C69E900EC96EFF0E9EB602D0E82EFCD71A
:106130009E96C69E000EC96EFF0E9EB602D0E82E39
:10614000FCD79E96C69E000EC96EFF0E9EB602D06C
:10615000E82EFCD79E96C69E000EC96EFF0E9EB618
:1061600002D0E82EFCD79E96C69EC952FF0E9EB660
:1061700002D0E82EFCD7C9CF2DF59E96C69EC952F7
:10618000FF0E9EB602D0E82EFCD7C9CF2EF5898A25
:10619000120018EC28F0B5C5E8FFD70802E318ECA8
:1061A00028F0B5C5E8FFC80802E318EC28F0B5C52B
:1061B000E8FFB90802E318EC28F0B5C5E8FFAA0823
:1061C00002E318EC28F0B5C5E8FF9B0802E318ECE1
:1061D00028F057EC2BF01EEC2FF0F29CF29E8B94E3
:1061E000C69AC2909482948C720ED36ED3A4FED7BA
:1061F00089968A909390FF0EE8CF00F0E82EFED7A4
:10620000002EFCD78150F294F29A9E909D909E921F
:106210009D92F298F292F290F286F28E0300FF00C5
:10BF0000E844F926000C160C2B0C3F0C520C640C68
:10BF1000760C860C960CA50CB30CC10CCF0CDC0C6B
:06BF2000E80CF40C000C1B
:0200000400F00A
:0100C800FE39
:00000001FF
